:020000020000FC
:0200000012C02C
:02000C007DC6AF
:10002400F3C60FED01BB0FEF02BB0FE304BB00E00F
:1000340005BB01E20ABB0FE00BBB0FEF07BB0FEFE1
:1000440008BB0FE50DBF04E00EBF00E010E021E0A7
:1000540031E040E050E060E070E080E090E0009348
:1000640008010093090100930A0100930B01009316
:100074000101009302010093030100930401009322
:1000840005010093060100931201009313010093EC
:1000940014010093150100931601009317010093B6
:1000A400190100930D0100930F01009310010093B7
:1000B4001B0100931C01009322010093250100936E
:1000C400240101E00093180100932301009300012F
:1000D4000093070100930C0100930E0100931D018E
:1000E40000931E01009321010093200103E000937B
:1000F4001F010AE00093110100E009BF08E002BDFE
:1001040003E003BF00E00FBD0BE00EBD00E00BBD3C
:1001140009E20ABD0BE005BD05E603BD01E809BF20
:1001240002B50830E9F708B70660076008BF00E8C1
:1001340008B9789409B30071003161F400E00093C8
:10014400250101E809BF00E405BF78948895000003
:10015400F894F0CF0BB300720032E9F001E00093A1
:10016400250100911E01003031F002B501FDFDCFE3
:1001740000E000931E010FE305BB0FEF02BB0FEF7E
:1001840008BBD89A00E809BF00E705BF78948895B2
:100194000000F894CFCF01E0009325010FE305BBE5
:1001A4000FEF02BB0FEF08BBD89A01E809BF00E4C8
:1001B40005BF789488950000F894BCCF213051F0A5
:1001C400223099F02330F9F0243049F12530A9F197
:1001D4002630F9F1042F7ED602BB00910C017AD6A9
:1001E4000F7D08BB01E005BB0895052F73D602BB44
:1001F40000910D01003011F06DD601C00FEF08BB66
:1002040002E005BB0895062F65D6D89802BB00917D
:100214000E0160D60F7D08BB04E005BB0895072FCF
:1002240059D602BB00910F01003011F053D601C022
:100234000FEF08BB08E005BB0895082F4BD6D898EC
:1002440002BB0091070150D60F7D08BB00E105BB3E
:100254000895092F003011F03DD601C00FEF02BB05
:100264000091070141D618BB00E205BB0895213077
:1002740051F0223081F02330B1F0243001F12530E7
:1002840041F1263091F1042F25D602BB07EA08BBC1
:1002940001E005BB0895052F1DD602BB08E208BB8B
:1002A40002E005BB0895062F15D6D89802BB00912D
:1002B400080110D608BBC59804E005BB0895072FB4
:1002C40009D602BB0091090105D608BB08E005BBAD
:1002D4000895082FFFD5D89802BB00910A01FAD5DA
:1002E40008BBC59800E105BB0895092F003011F043
:1002F400F1D501C00FEF02BB00910B01003011F0EA
:10030400E9D501C00FEF08BB00E205BB0895213019
:1003140051F0223091F02330D9F0243021F12530EE
:1003240069F12630B1F1042FD5D502BB009101014A
:10033400D1D508BB01E005BB0895052FCBD502BB81
:1003440000910201C7D508BBC59802E005BB08951A
:10035400062FC0D5D89802BB00910301BBD508BBBA
:1003640004E005BB0895072FB5D502BB0091040135
:10037400B1D508BBC59808E005BB0895082FAAD5D8
:10038400D89802BB00910501A5D508BB00E105BBC7
:100394000895092F003011F09DD501C00FEF02BB65
:1003A4000091060197D508BBC59800E205BB0895E6
:1003B400213051F0223081F02330C9F02430F9F09B
:1003C400253041F1263071F100910C0183D508BB31
:1003D400C59801E005BB089500910D01003011F0AE
:1003E40079D501C00FEF08BB02E005BB0895009169
:1003F4000E0170D508BBC59804E005BB08950091B3
:100404000F01003011F066D501C00FEF08BB08E002
:1004140005BB08950091070167D508BBC59800E1A5
:1004240005BB0895009107015FD518BB00E205BB29
:100434000895213051F0223091F02330C9F0243056
:1004440001F1253031F1263079F1042F43D502BB77
:10045400009110015AD508BB01E005BB0895052F92
:1004640039D502BB07EA08BBC59802E005BB08956D
:10047400062F30D5D89802BB08E208BB04E005BBC0
:100484000895072F27D502BB0FEF08BB08E005BB73
:100494000895082F1FD5D89802BB009121013FD59C
:1004A40008BB00E105BB0895092F003011F012D5F7
:1004B40001C00FEF02BB0091210131D518BB00E24E
:1004C40005BB0895213051F0223071F0233091F0B2
:1004D4002430B9F02530D9F0263001F1042FFAD4B4
:1004E40002BB01E005BB0895052FF4D402BB02E072
:1004F40005BB0895062FEED4D89802BB04E005BBD3
:100504000895072FE7D402BB08E005BB0895082F20
:10051400E1D4D89802BB00E105BB0895092F00304F
:1005240011F0D8D401C00FEF02BB00E205BB08955F
:100534002130B1F4042FCED402BB00911201CAD4ED
:1005440010911901113021F41091110110FD0FEFD8
:100554001091180110FD0F7D08BB01E005BB089543
:10056400223091F4052FB6D402BB00911301B2D40A
:1005740010911901123021F41091110110FD0FEFA7
:1005840008BB02E005BB08952330B9F4062FA2D4BA
:10059400D89802BB009114019DD410911901133015
:1005A40021F41091110110FD0FEF10911A0111FFA8
:1005B4000F7D08BB04E005BB0895243091F4072F98
:1005C40089D402BB0091150185D41091190114300E
:1005D40021F41091110110FD0FEF08BB08E005BBD9
:1005E40008952530B9F4082F75D4D89802BB00912A
:1005F400160170D410911901153021F410911101D4
:1006040010FD0FEF10911A0111FF0F7D08BB00E1DF
:1006140005BB0895092F003011F05CD401C00FEF21
:1006240002BB0091170156D410911901163021F420
:100634001091110110FD0FEF08BB00E205BB0895F6
:10064400213051F0223079F02330A1F02430B9F078
:100654002530D1F0263001F100911F013BD408BBB5
:1006640001E005BB08950091200134D408BB02E0E9
:1006740005BB08950DEF08BB04E005BB08950FEF1B
:1006840008BB08E005BB0895009107012DD408BB01
:10069400C59800E105BB08950091070125D418BB56
:1006A40000E205BB089543954A30E0F040E05395DD
:1006B4005630C0F050E063956A3098F060E073956E
:1006C400763078F070E08395DFD08A3010F080E0E7
:1006D4009395843030F0923020F080E090E003D0A5
:1006E40055D05FD0089500910E01039500930E013B
:1006F4000A3040F000E000930E0100910F010395D1
:1007040000930F0173D000910F01011748F16ED0CF
:1007140010910E01101720F101E000930E0100E08A
:1007240000930F0100910C01039500930C010A3012
:1007340040F000E000930C0100910D01039500933B
:100744000D0100910D01013058F000910C010330AE
:1007540038F001E000930C0100E000930D0101D09A
:10076400089500911F01039500931F010A3068F05A
:1007740000E000931F0100912001039500932001E4
:100784000A3018F000E00093200108950091070159
:10079400039500930701083018F001E00093070166
:1007A400089500911001003001F1013031F003305F
:1007B40021F0009107010630C0F4009108010617EA
:1007C400A1F400910901071781F400910A010817A7
:1007D40061F400910B01091741F4DD9A00911001B5
:1007E400013019F400E000931001089500910C0108
:1007F40010910D01103019F0039503950395013004
:1008040081F0023089F00330C1F00430C9F00530C2
:10081400D1F00630D9F00730E1F00830E9F00930C2
:10082400F1F013E002E008951DD0103019F412E045
:1008340009E0089513E000E0089513E002E008954C
:1008440013E001E0089513E002E0089513E001E0ED
:10085400089513E002E0089513E002E0089513E020
:1008640001E008951091200100911F0111701130D1
:1008740011F40395039511E0003029F0043019F0C8
:10088400083009F010E0089500912101003071F161
:1008940000910F01003051F1013041F1033021F09A
:1008A40000910E01053010F1009107010730F1F4B9
:1008B40000910C01033029F000910C01003041F04B
:1008C40015C0823099F4903089F483E090E0089563
:1008D40000912201013051F0833041F4903031F421
:1008E40082E090E001E000932201089500E000938B
:1008F40022010895009112010A95009312010F3FFD
:1009040099F509E000931201009113010A950093EF
:1009140013010F3F49F505E0009313010091140101
:100924000A95009314010F3FF9F409E000931401B0
:10093400009115010A95009315010F3FA9F405E0F4
:1009440000931501009116010A95009316010F3FBB
:1009540059F409E000931601009117010A950093D8
:1009640017010F3F09F401D0089500E00093170127
:1009740000931601009315010093140100931301D1
:100984000093120101E000931801DD9A089500918B
:100994001C01003019F00A9500931C0110911B01F1
:1009A40009B30E7000931B01101781F010911C0104
:1009B400103061F401FF05C002FF05C003FF05C04C
:1009C40005C0CDD003C02ED001C091D115E001FFE8
:1009D40010931C0102FF10931C0103FF10931C01D0
:1009E4000E3029F0109126011395109326011091D1
:1009F4001C01103019F410E0109326011091260107
:100A0400143679F41CE51093260101FF05C002FF9A
:100A140005C003FF05C005C0A2D003C003D001C0B8
:100A24006FD108950091250100FD0895313071F0D2
:100A3400323069F0333061F0343059F0353051F0F0
:100A4400363049F0373041F0383039F007C00EC045
:100A54001BC02FC04CC054C060C07FC00091230194
:100A6400053019F0039500932301089500911801AE
:100A740001E00093180100911901003009F407E026
:100A84000A9500931901089500910001023069F05C
:100A940000E000930101009302010093030100931D
:100AA4000401009305010093060101E00093000195
:100AB400089500910A01039500930A010A3040F059
:100AC40000E000930A0100910B01039500930B01D0
:100AD40000910B01023048F000910A01043028F023
:100AE40000E000930A0100930B015BDE089500917E
:100AF40021010395023008F000E0009321010895DC
:100B040083958A3010F080E09395843020F0923001
:100B140010F080E090E045DE089500910E01039509
:100B240000930E010A3040F000E000930E010091A2
:100B34000F01039500930F0159DE00910F01011776
:100B440058F054DE10910E01101730F001E00093BC
:100B54000E0100E000930F01089518DE089500913E
:100B6400250100FD0895313071F0323069F03330E1
:100B740061F0343059F0353051F0363049F03730C7
:100B840041F0383039F007C00EC05BC062C077C096
:100B94007FC08DC0AAC000912301003019F00A95CE
:100BA40000932301089500911901003061F0013090
:100BB40091F00230C9F0033001F1043039F105300D
:100BC40071F10630A9F1009118010A9509F402E0C7
:100BD4000093180108950091120103950A3008F05A
:100BE40000E000931201089500911301039506306B
:100BF40008F000E000931301089500911401039597
:100C04000A3008F000E000931401089500911501E2
:100C14000395063008F000E0009315010895009153
:100C2400160103950A3008F000E0009316010895B8
:100C34000091170103950A3008F000E000931701B2
:100C44000895009100010A9509F402E0009300015F
:100C54000895009108010395009308010A3068F093
:100C640000E0009308010091090103950093090134
:100C7400063018F000E00093090193DD0895009117
:100C840010010395043008F000E00093100108956A
:100C940063956A3028F060E07395763008F070E070
:100CA40040E050E00AE0009311017BDD08950091DB
:100CB4000C01039500930C010A3040F000E000930E
:100CC4000C0100910D01039500930D0100910D019C
:100CD400013050F000910C01033030F001E000933A
:100CE4000C0100E000930D0108953BDD08950BB362
:100CF4000072003219F03A9509F435E0DD98089550
:100D040038E0089500911D010A9509F40AE0009362
:100D14001D010A3019F0063039F00BC016E613BD78
:100D240001E000931E0105C015E613BD01E0009328
:100D34001E01009111010A9579F4B5DC09E2041B46
:100D4400041B0ABD00E00DBD00E00CBD00911801BC
:100D5400023009F4CFDD0AE0009311010091000193
:100D64000230E1F5009101010395009301010A307D
:100D7400A8F100E0009301010091020103950093A2
:100D840002010A3058F100E00093020100910301CE
:100D9400039500930301063008F100E0009303017A
:100DA400009104010395009304010A30B8F000E0B7
:100DB4000093040100910501039500930501063099
:100DC40068F000E00093050100910601039500938B
:100DD40006010A3018F000E00093060100911A01A0
:100DE4000A9509F405E000931A0110E00BB30072B0
:100DF400003239F400911A0101FD03C010E48D9A08
:100E040001C08D981FBD18950091240110912301F4
:100E1400103051F0113051F0123051F0133051F0C4
:100E2400143051F0153051F018E909C01CEC07C01A
:100E340016EE05C013EF03C019EF01C01CEF01301B
:100E440011F0003089F00FEF011B17E6101B0FEFB4
:100E5400011B02BF00E00093240100912501013031
:100E640081F000E005BB189512BF01E00093240156
:100E74002A9511F426E08BDD00912501013009F05B
:100E840001D0189500E005BB0FEF02BB0FEF08BBC4
:100E9400D89A313071F0323071F0333071F034302F
:100EA40071F0353071F0363071F0373071F0383020
:100EB40071F084D90EC03CDB0CC029DA0AC0D7D942
:100EC40008C0B7DA06C0FEDA04C072DA02C0B8DBC2
:100ED40000C008950A3008F00AE0FFE0E6E3E00FFE
:100EE4000027F01F04910895083008F000E0102F47
:100EF400FFE0E2E4E00F0027F01F0491FFE0EAE4E2
:100F0400E10F1127F11F14910895043008F004E053
:100F1400FFE0E2E5E00F0027F01F049108950030A0
:100F240011F0013019F007EF17EF089503EE18E2FE
:100F34000895A0F96470393222F820307F7F7F63EE
:100F44002727272863267F2CA132A62C326BF7F99A
:040F540032F87F7F71
:00000001FF
